:020000001428C2
:080008009800030E831297001B
:10001000393081000B1104309F061F1D990A170EFD
:100020008300980E180E090083128501860183163D
:100030000630810083123930810020308B0020305F
:1000400084008001840A041F2128041E21288316AD
:100050003F30850081308600831205309D000130DD
:1000600093008B179F0013089F04A030CE0001302F
:10007000910049309000F3204C0886004A08850022
:100080008316050894000608930083121409CA0514
:1000900005091405CA041309CC0506091305CC0487
:1000A00001308D008E018C014A190C1440180C147B
:1000B000C0188C010130930041309500403096000B
:1000C00001309200CD218E018C014A1D0C14233089
:1000D0009300423095004030960002309200CD21CE
:1000E0008E018C01C01C0C14C01A0C144A198C010E
:1000F0000230930046309500403096002030920048
:10010000CD218E018C01C0180C14C0198C01063051
:100110009300433095004030960004309200CD218A
:100120008E018C0140190C14053093004430950069
:100130004030960008309200CD218E018C01C0180D
:100140000C14FA3093004530950040309600103082
:100150009200CD218E018C0140180C1403108F0DDC
:100160000C180F144C308400203092008A218C012E
:100170000F180C1403108F0C4C3084004030920088
:100180008A218E018C01C01A0C14401A8C014C304B
:100190008400043092008A218E018C0140180C14D6
:1001A0004C308400023092008A218E018C0140196B
:1001B0000C14401A8C0103108F0D0C180F144C30C6
:1001C0008400083092008A218C010F180C1403104F
:1001D0008F0C4C308400103092008A218E017F30C9
:1001E000CE051F10372864001A081902031DFB28CA
:1001F0009F19F3283B29031C01309B0719089A001B
:100200009F1F08294730840000080319082980032C
:100210001F1F22291B08053C031912291B080A3C31
:10022000031D2229013094009C0A1C182029033048
:1002300094000A301C02031C20299C010730940002
:100240001408CF060A301B02031C3B299B001D0823
:100250009400140F2C293B291F1E000041309407E5
:1002600084000008031935298003040814020319C7
:100270003B29840A312908000C080D0508000310E9
:100280000E0D0C048E0008000E0801398C054B2958
:100290000E0801398C0403108E0C080013081E048C
:1002A0005A293C21031957291E0812045A291E08ED
:1002B000920912059E009200920C9403031C662979
:1002C000031963295C2901308D0008008D010800A5
:1002D0003C2103198929160884001218802903106B
:1002E000120C000503197729120880047A291209D3
:1002F000800589290310120C9400140980058929AE
:100300008403801F87298013840A00148929840AA2
:10031000001008003C2103199029000812049329B9
:1003200000089209120580000800100884000008E7
:100330001105031D9C2968211E2208003C21031978
:10034000080000081204800008003C21031908007E
:1003500000089209120580000800100884000008B7
:100360001105031DBB293C210319BB291608840074
:1003700000081204C029160884000008920912051A
:1003800080001E22080010088400000811050319CF
:10039000BB293C21031DBB29B62910088400000895
:1003A0001105031DD7293C210319DA29E1293C2134
:1003B000031DE6299301160884000008920912051E
:1003C00080001508840013088000F02915088400B7
:1003D0000008031DF029160884000008120480009C
:1003E0001E2208001608840000081205031D0F2AAB
:1003F0003C2103190F2A1008840000081105031D71
:100400000F2A15088400800A0008130203190A2A1B
:1004100003180F2A160884000008120480001E2208
:1004200008003C21031908001608840000089209FE
:10043000120580001508840080010800100884005F
:100440003C21031D282A91090008110591092A2A37
:100450000008110480000310910D031C322A0130A2
:100460009100900A08000A3092003922920B352A36
:1004700008007F3093007F309400940B3D2A930B4B
:040480003B2A08000B
:02400E00F23F7F
:00000001FF
